:10014000021D800A0A5052494E540D0A80140A506A
:1001500052494E540D0A801E205052494E542022BE
:10016000544154544C4554414C45204D4F44454C0A
:100170002023223B0D208028105052494E54204D00
:100180004F44454C0D1080320A5052494E540D0ACE
:10019000803C225052494E5420222020532F4E2082
:1001A000222C20534E25313030303030303030303A
:1001B0000D2280462A5052494E542022284329209D
:1001C00031393838204F4E53455420434F4D505508
:1001D00054455220434F52502E220D2A80500A502F
:1001E00052494E540D0A805A2F5052494E542022E3
:1001F0005454424153494320222C564552532F31E7
:1002000030302C222E222C2330322C5645525325AE
:0D0210003130300D2F8064084E45570D0829
:10C000008E00FFBDF5DF8621BDF8F3BDC0C842C07C
:10C010002743C03044C03946C07B4DC12B50C29F1E
:10C0200052C27653C0AA00BDF8F3717F147EF9495D
:10C03000BDF8F3BDF5DF7EC6FEBDC0E33CBDFA77BB
:10C04000BDF918383CC610A600BDFA7CBDF91C0825
:10C050005A26F4BDF91838C610A60081202C028695
:10C060002E817F2F02862EBDF8F3085A26EBBDF5F0
:10C07000DFBDC128812E26C47EC000BDF8F3BDF906
:10C080001CBDC0F6183C862CBDF8F3BDC0F6DD56CD
:10C09000862CBDF8F3BDC0F637BDF5DF3238A700FA
:10C0A000089C5626F9A7007EC000BDC0E3BDFA7704
:10C0B000BDF918A6009753BDFA7CBDF918BDC0F6AE
:10C0C000E700BDF5DF0820E5383CBDC128A1002709
:10C0D000096D0027F308080820F3333336EC011804
:10C0E000326E00BDF8F3BDF91C7F00527F0053BDD6
:10C0F000C0F6187EF5DFBDC128812E26037EC00064
:10C10000810D2603DC5239803025EB810A25088019
:10C110000725E3811024DF9746BDFA84DC5205052C
:10C120000505DB46DD5220CE7EF8B6BDF8F3BDF541
:10C13000DFBDF88126FB71F8175FF740005CC10294
:10C1400027057C001720F371F8175FF140002738AE
:10C15000B64000363771F817CEC1754FBDF4603266
:10C160008A30BDF8F3CEC17D4FBDF460328A30BD58
:10C17000F8F37EC0003A2042414E4B200020524549
:10C1800041445320415320005CC10227057C001725
:10C1900020B971F817CE4002EF001805847F8B405C
:10C1A000188C400026F2CE4002AC002743DF46EE5A
:10C1B00000DF4871F817BDF5DFCEC1E14FBDF46077
:10C1C0009648BDFA7C9649BDFA7CCEC1E64FBDF4D7
:10C1D000609646BDFA7C9647BDFA7C71F8177EC022
:10C1E0000053454520002041542041444452200042
:10C1F0001805847F8B40188C400026AD8601974639
:10C2000071F81796179A469717CE40004F5FED00CA
:10C21000EC00261E4353ED00A300261F08088CC027
:10C220000026EB7C00469646810226D771F8177EE1
:10C23000C000CC0000ED00EC002007CCFFFFED00BB
:10C24000EC003C373671F817BDF5DFCEC26B4FBD41
:10C25000F460323318BDFA778640BDF8F3383CBD40
:10C26000FA7738EC004353ED0020F842495420455A
:10C2700052524F522000BDF8F3BDF5DF4F36323633
:10C28000BDF65FDE56BDFA77BDF918324C368140F7
:10C290002709840726E8BDF5DF20E3327EC000BD14
:10C2A000F8F3BDF5DF7F0053BDC0F6C43F37BDF9DD
:0DC2B00018BDC0F6DD5632BDF6AF7EC000F1
:10C4000000000030303030303030303030300D54BB
:10C410004154544C4554414C45204D4F44454C20CB
:10C420003220202843292031393838204F4E5345B7
:10C430005420434F4D505554455220434F52502E97
:10C440000D4C495354CB15545952554ECAB3505202
:10C45000452A52554ECAAC462452454D494E44CF0A
:10C4600091465245D73B414F4E454F4ED7E3414150
:10C4700041454F4646D7DE42424E455854C9315495
:10C480004F4C4554CE785641524946CDBC4E4F5440
:10C4900045474F544FCAFD454E474F535542CD6710
:10C4A0005352455455524ECD90464F52C8A9474518
:10C4B000544255525354CE885853544F5245CECBC4
:10C4C0004150534554D392564150434C52D3FC549F
:10C4D0004553444FDAC731313143414C4CDBF232E2
:10C4E00032434F554E54DD2445534C454550D314EB
:10C4F000525550524F47DB8A5855474554D4E9446A
:10C5000046544F4E45D75652535553454E44D4602A
:10C510002F4F4E455252D63F2341534DDE944A4E43
:10C520004B52454DCDAD41524B5052494E54CC46E5
:10C5300053584D4954D80B574F53544F50CAA654D3
:10C540004F4954455854D65F4F4F54455854D6F32D
:10C55000475354494D45D828405254494D45D987F1
:10C56000405653544F5245DC7556474554DCAF3363
:10C5700033494E505554CDE138585348414B45D777
:10C58000EE4F46464C44D156454F4E4C4F4144DD4C
:10C590006244494DDCE15245414E4557CA924F4CE9
:10C5A00044434F4EDD03444545CE72544FC8CC46FC
:10C5B000524F4DF2C253544550C8E14154C8E7436D
:10C5C00048414EE5565459474554E59226474F5049
:10C5D000494EE610544845534449E98220202050F2
:10C5E0004552494F44EA69414253E541424545536A
:10C5F0005152E69147415454454D50E746484953FE
:10C60000494EE8074F46464153494EE8734E55435D
:10C610004F554E54E9D5454C4F47EB26494E4745BB
:10C620005850ECE1495245424154E72B544F505683
:10C63000455253E9675A59534EE97350495A454D8B
:10C640004F44454CE95E53E50D3DE393252F2F2ADA
:10C65000343E3DE3642F233C2F3E3CE36F7E2F2A84
:10C660003C3C3EE36F2B3D2D3E3EE381454E442E48
:10C670002E3C3DE38A3F2F3E3E3CE39A3C3E3C3E0F
:10C680003CE3A18EBFFF7F00760E86FF9791BDF839
:10C6900054861A97111A1ABDF8544FCE738C6F0036
:10C6A000088C73A226F87F00B37F00B4CC0C00FD89
:10C6B00072887F00B57F006A7F0076860AB7B59AD8
:10C6C000CC1770DDAF8639979F9797979497A5976A
:10C6D000A897A2867E97ABCCF8F3DDACCC0000DD4A
:10C6E0009ADD9C7F0077BDF5DF86FF978C979E7F54
:10C6F00000927F00B67F00937EC82C4F4B0D8EBFFB
:10C70000FF86FF979E860AB7B59A7F00817F008CCF
:10C71000BDF5DFCEC6FB4FBDF460CEC721FF738CE5
:10C72000CE0000FF7394FF738E863EBDF8F34FCEAC
:10C73000B294BDF370083CCEB294865CBDEDE726A2
:10C740001EBDE2DFFC721893522607FC721A935446
:10C7500027033820D4865CBDEDE727037EF2C2189C
:10C7600038DF5618BDEE6CDC56DD4EBDEDF7DC5201
:10C770002634DC54261B8627BDEDE727AC7EC85B3C
:10C7800045444954494E472044495341424C45444D
:10C790000D7D0092270DCEC7804FBDF460BDF5DF43
:10C7A0007EC7294D2A06CC00087EEF0B0909098AAD
:10C7B00080ED00DF46DC4E9346E702DE4E09E700DF
:10C7C000BDF3DD2705FF73AE201BFF73A6FF73AE1D
:10C7D000FC73A2FD73A8BDF401FF73A4BDF551FC69
:10C7E00073A6FD73A2DC4E9346C10526037EC729BE
:10C7F000FE73A2FF73AAF373AAFD73AC188CB28FF9
:10C800001823037EF367FD73A2BDF56AFC73AEFDCA
:10C8100073A6DC4EFD73A8DC46FD73A4BDF5517E06
:10C82000C729CE01006F000926F8203AFEB5CD8C4D
:10C8300030392722B6C42E815326E7CE0142FF733A
:10C84000A4CE73D2FF73A6FC0140FD73A8BDF551C1
:10C85000FC73A6FD73A27ECAAF0000CCC859FD735D
:10C860008CCCC441DD520908A600B1C42B27F8DFE7
:10C8700046A6003CDE52E6002B2811270B18C30009
:10C880000818DF5220F0DE4A08E600DF4A38083C8C
:10C89000E10027F2C180240838DE463CDE5220DD6C
:10C8A000DE4A08A60038363739BDF5AABDF27ADC73
:10C8B00052FD7394B6C42C814F2709FC73948300F6
:10C8C00004FD7394CCC5ABDD527EC866BDE2DFDCEF
:10C8D00054FD7398DC52FD7396CCC5B5DD527EC80D
:10C8E00066BDE2DF7EC8F0CC0001DD545F4FDD5253
:10C8F000DC52FD739ADC54FD739CFC738CFD739EBB
:10C90000FF73A030200518C3000E18EC00271C1878
:10C91000BC73941826F0FF73AA18C3000EFD73AC05
:10C9200030FF73AEBDF56AFE73AC35FE73A07EEDCD
:10C93000FEBDEE0424037EF2C2FD73903CFE7394B0
:10C940002604387EF2C2BC7390270738BDF5837E7B
:10C95000C93CEC02F3739CED02EC00F9739BB973D4
:10C960009A295BED00FC739A2B267D73962A066D3F
:10C97000002A4D20046D002B39EC0018BC7396255D
:10C9800031263D18EC0218BC739825262724203048
:10C990007D73962B066D002B2720046D002A13EC67
:10C9A0000018BC73962519260918EC0218BC739858
:10C9B000250E38FC739EFD738CFE73A02006ED00DF
:10C9C00038BDF5837EEDFEBDE2DFDC522605DC548A
:10C9D0004D2A09CC00087EEF0B7EF2C23637862C3A
:10C9E000BDEDE726F4BDE2DFDC5226E7DC544D2B3B
:10C9F000E23332DD48DC54934825D83CFE738CEC9E
:10CA000000847FDD502733189C48252E9C54270234
:10CA10002428BDF5DFCECA204FBDF460387EC6FEA7
:10CA200043414E4E4F5420455241534520435552A9
:10CA300052454E54204C494E450DDE54DF52DE48DF
:10CA4000DF54CE73D2BDF3EF2404387EEDFEFF73C6
:10CA5000A6DC52C30001DD54BDF3EF2408FC73A62D
:10CA6000FD73A22012FF73A4FE73A2FF73A8BDF58D
:10CA700051FE73A6FF73A2DE5027CFDF54CE73D2D0
:10CA8000BDF3EF080808A600810D27BF813A27BB38
:10CA900020F3BDEDF7810D2707813A27037EC9C733
:10CAA000CC73D2FD73A2BDF2B77EC6FEBDF2B786CF
:10CAB000FF2004BDF2B74F978C7F0081CE73D27FE9
:10CAC00000547F0055BDF3EF24037EC6FEFF738C38
:10CAD00096B5271BBDF8F3EC00847FDD547F005230
:10CAE0007F005386019745BDF49B863EBDF8F30851
:10CAF0000808BDF5F0CCC479DD527EC866BDE2DF22
:10CB00003CBDF2B7BDF414270738CC00157EEF0BFF
:10CB100032327ECACDBDEE0424037ECBB23CFD731F
:10CB2000AA18EC00DD64EC02DD66CCEFD5DDAC3894
:10CB30007F00547F0055862CBDEDE7260DBDEE6CC1
:10CB4000DC522706CC00087EEF0BDC542BF6363780
:10CB500096442729862CBDEDE7270A862DB1C42EE1
:10CB6000BDEDE72613BDEE6C96442711DC5226D4AA
:10CB7000DC542BD0DD5E200ACC00002003CC7FFFEC
:10CB8000DD5E3332DD543CBDF3DD2512BDF52CBD39
:10CB9000F3EF250AEC00847F935E27F025EEFE7309
:10CBA000AADC64ED00DC66ED02CCF8F3DDAC387E87
:10CBB000C6FEBDEE6CDC522706CC00087EEF0BDC17
:10CBC000542BF6363796442729862CBDEDE7270AE5
:10CBD000862DB1C42EBDEDE72613BDEE6C9644271D
:10CBE00011DC5226D4DC542BD0DD5E200ACC0000B0
:10CBF0002003CC7FFFDD5E3332DD5496763686012E
:10CC000097763CBDF3DD2517BDF52C7D0093262AD4
:10CC1000BDF3EF250AEC00847F935E27EB25E9380E
:10CC20003284019776863BBDEDE7260BBDF8B681D1
:10CC30001327F9811127F57EC6FE383284019776D5
:10CC4000BDF8547EC6FE863BBDEDE726037EEDFEB5
:10CC5000860DBDEDE7270C863ABDEDE727058D0A69
:10CC60007EEDFE09BDF5DF7EEDFE86019745BDF444
:10CC70007427698623BDEDE72639C600A6008130FA
:10CC80002602C680D745BDE2DF9655847F9A459738
:10CC9000458648C610A10027138642C602A1002778
:10CCA0000B8651C608A1002703C60A0908F7B59AE2
:10CCB0007ECCDCA600815C260A08BDE2DF96559D8D
:10CCC000AB2019867BBDEDE7260CBDCD01867DBD71
:10CCD000EDE726252006BDE2DFBDF49B862CBDEDE9
:10CCE000E7278B863BBDEDE7260139860DBDEDE7D5
:10CCF000270A863ABDEDE727037EF2C2BDF5DF09BC
:10CD000039BDE2DFBDCF6ADC523637DC54363786B8
:10CD10002CBDEDE726E3BDE2DFBDCF6A3332DD484F
:10CD20003332DD469352250E2706CC00167EEF0BDC
:10CD3000DC54934825F4BDCD50BDF040BDCD509D91
:10CD4000ABDC46935225EF2606DC54934824E739A2
:10CD50003CDE463CDE483CDE64DF46DE66DF4838CB
:10CD6000DF6638DF643839BDF5AABDE2DFBDF2B752
:10CD70003CBDF414270738CC00157EEF0B18FE736A
:10CD80008C3CFE738E3C7F7394BF738E187ECACD2D
:10CD9000BDF2B7FC738E26037EF2C2BE738E38FFDF
:10CDA000738E38FF738C38BDF5837EEDFEFE738C79
:10CDB0007F00547F0055BDF4017ECAC8BDE2DFDCB0
:10CDC000522604DC5427037ECAF2BDF40B25037EF1
:10CDD000CACD7EC6FEBE739238FF738C3838BDF55F
:10CDE000DF3CBDF4742609BDEE04DD542568202324
:10CDF0003CBDEE04DD5424037EF2C2A600B1C42D76
:10CE000097454FA70038BDF460964509A700863ABC
:10CE1000BDF8F33CFE738C3CCEFFFFFF738CBF73F9
:10CE200092DC543736863ACEB394BDF370CEB394C9
:10CE3000A600810D2606A7018630A700BDE2DFBD52
:10CE4000EDF7810D268F380FDC54ED02DC52ED003A
:10CE50000E38FF738C3832B1C43132863BBDEDE7FA
:10CE60002703BDF5DF862CBDEDE726037ECDE17EF1
:10CE7000EDFEA600810D270ABDF27A862CBDEDE7F6
:10CE800027F67EEDFE7EF2C2BDCF51862CBDEDE7CA
:10CE900026F3BDE2DF3CDE522609DE5427058C0076
:10CEA00009250738CC000B7EEF0B18D7467F0047CB
:10CEB000D6474FC3E58A18E600BDF71217BDEFD578
:10CEC0007C00479647914626E7202CBDCF518631FE
:10CED0009762862CBDEDE7261D8623BDEDE7263142
:10CEE000A600088132270B81342707813127037E72
:10CEF000F2C2976220DC3CFE73AAB6C42D814E2795
:10CF000004DC422002DC66ED02DC64ED00387EEDDC
:10CF1000FEBDEDF78127270481222610CCEFD5DD59
:10CF2000ACBDCC6ACCF8F3DDAC7ECEF6BDE2DFD68C
:10CF300062C134260C9652BDEFD59653BDEFD52075
:10CF400004C13226059654BDEFD59655BDEFD520C8
:10CF500081BDEE042511FD73AA3CFE73AAEC00DD31
:10CF600064EC02DD6638397EF2C2CC0000DD46CCCE
:10CF70008000D39CDD48DC46D99B999A9352250BBF
:10CF80002608DC4893542503270139CC00167EEF90
:10CF90000B3CFC73A28373D22604387EEDFE188C02
:10CFA0003EBF2534CECFAE4FBDF4607EC6FE50529C
:10CFB0004F4752414D20544F4F2042494720464F42
:10CFC0005220524F4D2028313633383220425954A6
:10CFD0004553204D4158290018C30142FD73D0CE5E
:10CFE000D2E74FBDF460BDF5DFCE17701ABDF87CF7
:10CFF000260D0926F7CED2F74FBDF4607EC6FEBDE2
:10D00000F8B6811826037EC6FE8115268DCEB601A0
:10D01000DF5286019755FC73A2DD4ACC8D70DD4C42
:10D02000CE73D0BDD06038862BBDEDE73C260C4FCB
:10D030005FDD4CDD4ACEC000BDD0604FCED04BA6E8
:10D040000081242714BDD0E20820F43A303030307B
:10D050003030303030300D0A24BDD133387EEDFE13
:10D06000DF4E7F00467C0046089C4A270696468194
:10D070001026F2863ABDD0E27F00479646BDD0C169
:10D08000DC4ED34C37BDD0C132BDD0C14FBDD0C1B5
:10D09000DE4EA600BDD0C1089C4A27107A00462665
:10D0A000F14F9047BDD0C1BDD0B620B44F9047BD21
:10D0B000D0C1BDD0B639860DBDD0E2860ABDD0E262
:10D0C00039369B47DD47323644444444BDD0D432E0
:10D0D000BDD0D439840F8B30813A25028B07BDD067
:10D0E000E2393CDE52A7008CB680270608DF5238B2
:10D0F000393CCEB601DF524F97548601BDF8F39606
:10D1000055BDF8F343BDF8F3A600BDF8F39B549763
:10D1100054088CB68126F19654BDF8F3BDF8B6815B
:10D120001527CF810626CB811826037EC6FE7C00FC
:10D13000553839DE528CB681270B6F00088CB681CA
:10D1400026F8BDD0F18604BDF8F3BDF8B6811827E6
:10D15000DA810626DE39BDE2DFBDCF6ADC52DD644E
:10D16000DC54DD66862CBDEDE727037EF2C2BDE20E
:10D17000DFBDCF6ABDD2DC2406CC00167EEF0BB635
:10D18000C42E81532708DC529A40DA41DD5218DE62
:10D19000523CDE543C18862CBDEDE72707CC1770B7
:10D1A00036372020BDE2DFDC522706CC00177EEFA9
:10D1B0000BDC543637862CBDEDE72608BDEE042483
:10D1C000067EF2C2CC004EDD4E3332DD501838DF21
:10D1D0005438DF52183CDE4E8C004E260ACED2E781
:10D1E0004FBDF460BDF5DFBDD2002620DE4E8C00C1
:10D1F0004E260ACED2F74FBDF460BDF5DF7ED2CE0B
:10D20000DE501ABDF87C26030926F739BDF8B68131
:10D210001826037ED2CE811526CD8601974720346D
:10D220007C0047BDD200260D3338BDD2DC24037EFE
:10D23000D2AE7ED2CEBDF8B633388106271681181D
:10D2400026037ED2CE811527043C3720D6DF66D751
:10D25000657A0047BDD2DC254BDE663CD665377F5C
:10D26000005A7F005B8601BDF8F39647BDF8F34393
:10D27000BDF8F3BDD2DC2515965A8180271EBDF07E
:10D2800040BDF8F39B5B975B7C005A20E6965A8181
:10D290008027094FBDF8F37C005A20F1965BBDF85A
:10D2A000F37ED2208604BDF8F3BDD20026197300A8
:10D2B00064730065DC664353C30001DD66DC64C94A
:10D2C000008900DD642007BDF8B6810626D6DE4E53
:10D2D000DC64ED00DC66ED02387EEDFE9653906571
:10D2E0002604DC5493663957414954494E47204639
:10D2F0004F52204E414B004E414B204E4F54204642
:10D300004F554E44204245464F52452054494D45C5
:10D310004F555400BDE2DFDC522706CC00187EEFEB
:10D320000BDC54260D96431A914327FB4FDD6C7E90
:10D33000EDFEDD6E200108A600B1C43127F8813A68
:10D34000272C810D27283C20091ADC6C936E270BB3
:10D3500024097B401527F2387ECAF2DD6C38CC00F8
:10D3600000DD54BDF40B25037ECACD7EC6FE3C1AFB
:10D37000DC6E936C270925022AF5862ABDF8F3CEC8
:10D380000000DF6C387EEDFE9DA53838CC000C7EA9
:10D39000EF0BBDE2DFDC52270DCC000C7EEF0B3C27
:10D3A0008DE6387EEDFEDC544D26F4C10E24F0C12E
:10D3B00008241786805D2704445A20F9369A159769
:10D3C00015329A8B9720978B201EC00886805D2788
:10D3D00004445A20F9B1C43124024444369A0397D4
:10D3E00003329A8A9701978A862CBDEDE727A37EA0
:10D3F000EDFE9DA83838CC000C7EEF0BBDE2DFDCE3
:10D4000052270DCC000C7EEF0B3C8DE6387EEDFEF6
:10D41000DC544D26F4C10E24F0C108241886805D2A
:10D420002704445A20F9364394159715329A8B975E
:10D4300020978B2021C00886805D2704445A20F95C
:10D44000B1C43124024444364394039703329A8A88
:10D450009701978AC00E862CBDEDE7279F7EEDFED3
:10D46000BDD5D986809A8A9701978ABDEDF781222A
:10D47000270481272610CCD4BCDDACBDCC6ACCF807
:10D48000F3DDAC7EEDFEBDD619DC7B2604DC79270E
:10D490001BBDF040BDD4BCDC7B830001DD7BDC79AF
:10D4A000C2008200DD7926E9DC7B26E53CFE73AA1A
:10D4B000DC64ED00DC66ED02387EEDFE3CDE7D8C4A
:10D4C000011324010FBDD5D3717F03BDD5D3C60889
:10D4D000442505717F0320057280032000BDD5D34C
:10D4E0005A26ED728003380E39BDD5D9BDD61986BE
:10D4F0002CBDEDE727037EF2C2BDE2DFDC7B260711
:10D50000DC7926037ED4AC86FE948B9720978B869D
:10D510007EB7010CCCD57AFD010DDC522706CC007C
:10D52000257EEF0B0FDC42D354DD54DC40D95399F8
:10D5300052DD5296AE8900974E7F007FDF467F0016
:10D5400080DC7D83011325037A00800E01010F72B8
:10D5500001140E1A0F967F2616964E90AE251026B1
:10D56000EADC529340250826E2DC54934224DC7125
:10D57000FE140E86FF97807ED4AC71FE1496802731
:10D58000010ED61737C4F7D717DC7D04D37D18BD3D
:10D59000D5D5C68096150425070101BDD5D320F445
:10D5A00017DE46BDEFD5DC7B830001DD7BDC79C275
:10D5B000008200DD79DC7D04047B011526058300F3
:10D5C0000126F6DC792608DC7B260486FF977F336C
:10D5D000D7173BDE7D0926FD39BDE2DF3CDC52DD9D
:10D5E00046DC54DD48BDEF8ACC04B0DD53BDF0828B
:10D5F000DC52260CDE548C0FA024058C001E240A5D
:10D6000038CC00197EEF0B7EF2C218830007DD7D57
:10D6100038862CBDEDE726EF39BDE2DFDC52DD793F
:10D62000DC54DD7B862CBDEDE726DCBDEE0425D782
:10D63000FD73AA3C18EC00DD64EC02DD663839BDF0
:10D64000E2DFBDF2B73CBDF414270A387F0081CC7D
:10D6500000157EEF0BDF823886FF97817EEDFEBDE1
:10D66000CF51860DB773AC862CBDEDE72616865CD0
:10D67000BDEDE72636BDE2DF9655B773AC862CBD0F
:10D68000EDE727273C4FCEB394F673ACBDF372CED3
:10D69000B394A600B173AC270C08DF5238BDEFD5A8
:10D6A0003CDE5220EDBDEFD57ECEF7BDE2DFDC5291
:10D6B0002706CC001A7EEF0BDC54272ADC54DD52FF
:10D6C000BDF87C270FBDF8B636BDEFD532B173ACCF
:10D6D000271120EC1ABDF87C26E2DC52830001DD24
:10D6E0005226F17ECEF6BDF87C27F8BDF8B6BDEF28
:10D6F000D520F0BDCF51860DB773AC862CBDEDE7BC
:10D700002612865CBDEDE727037EF2C2BDE2DF96FE
:10D7100055B773AC3CBDF040B173AC2705BDF5E126
:10D7200020F33836863BBDEDE732270C810D260508
:10D73000BDF5DF2003BDF8F37ECEF6BDF2B7CCB267
:10D740008FB373A2DD547F00527F00538606974546
:10D75000BDF49B7EC6FEBDE2DFDC522706CC001B7B
:10D760007EEF0BDC54188C00DC1825F13637862C44
:10D77000BDEDE726E8BDE2DFDC5226E1DC542604FD
:10D780003232203A05DD5425D43332DD463C867EE4
:10D79000B70106CCD7C1FD010771FD03CC0000DD48
:10D7A00009DE46DF0B9608DF0B8601970F86089788
:10D7B000081ADC4626FB7F00088600970F387EEDAE
:10D7C000FE9608DE54270E09DF5488019708DC0B0B
:10D7D000D346DD0B3BDC0BD346DD0BDF463B86FF40
:10D7E0003620024F36BDF2B73297927EC6FEBDE2BA
:10D7F000DFDC522706CC001C7EEF0BDC542706DD55
:10D80000AF860120014F97767EEDFEA600812D2682
:10D810000DBDF88126FB86FF0897777EEDFE812BF4
:10D8200027037EF2C24F20F0B673B0BA73B1BA7359
:10D83000B4BA73B5BA73B8BA73B9BA73BCBA73BDB4
:10D84000BA73BEF673BF271FC12025028AFFBA73C1
:10D85000C0BA73C1BA73C2F673C3270BBA73C4BA22
:10D8600073C5BA73BE2706CC00267EEF0B7F004A35
:10D870007F004BFC73B2DD4CCC003CDD484F5FDDDC
:10D8800046DD52FC73B6DD54BDF1B6BDD96C4F5FB9
:10D89000DD46DD52CC0E10DD54FC73BADD48BDF11F
:10D8A000B6BDD96C4F5FDD465CDD52F673BF5ADD05
:10D8B00048CC5180DD54F673C7C1292404CB142011
:10D8C00008C050251AC1142416D75E54545CC107F1
:10D8D00025015A4FD348DD48F673C3C10D2506CC48
:10D8E000001D7EEF0BD7463CCED97BC103240DD65D
:10D8F0005EC1142707C40326037A00495F7A0046F5
:10D900002707EB0089000820F438D348DD48BDF133
:10D91000B6BDD96C4F5FDD52D65EDD54CC01E1DD82
:10D9200046CC3380DD48BDF1B6BDD96CBDEE0425D3
:10D930000E3C18DC4AED00DC4CED02387EEDFEDCDE
:10D940004CDD484FD64BDD465FDD52C664DD54BD2D
:10D95000F1B60FDC50DD42D64FD7418664D64A3D42
:10D96000DB4E8900D74097AE0E7EEDFEDC50D34CE7
:10D97000DD4CDC4ED94B994ADD4A391F1C1F1E1F56
:10D980001E1F1F1E1F1E1FBDEE043C24460F96AE19
:10D990009752DC40DD53DC4297550ED75ECC0064D5
:10D9A000DD485FDD46BDF082DC53DD5F9655976153
:10D9B0009651D65EDD544F5FDD52DD46C664DD48CC
:10D9C000BDF082DC549B61DD54DC5FC9008900DD61
:10D9D00052200918EC02DD54EC00DD52188C800056
:10D9E000250738CC001E7EEF0BCC0001DD46CC5164
:10D9F00080DD48BDF082DE543CDC4EDD52DC50DD83
:10DA0000544F5FDD46CC0E10DD48BDF082DC54FD86
:10DA100073BA5FFD73B8DC4EDD52DC50DD544F5FEE
:10DA2000DD46CC003CDD48BDF082DC54FD73B65FC2
:10DA3000FD73B4DC50FD73B25FFD73B038187F0026
:10DA4000527A00527C0052BDDAB0260A83016E245D
:10DA5000F3C3016E200883016D24E9C3016D3637DD
:10DA6000D652CB50C1642502C0644FFD73C65FFD22
:10DA700073C43332CED97B7F00547F00537C005374
:10DA800037E600BDDAB0260937D653C10233260186
:10DA90005C08D75533935424E4D3544F5CFD73BED4
:10DAA000D653FD73C25FFD73BCFD73C0387EEDFEBF
:10DAB00036965281142704840332394C3239CC0013
:10DAC000207EEF0B7EF2C2BDEDF781222704812775
:10DAD0002613BDDB76CCDB59DDACBDCC6ACCF8F3CC
:10DAE000DDAC7EEDFEBDE2DF18DE523CDE543C18BC
:10DAF000862CBDEDE726CDBDE2DFDC5226C0965474
:10DB000026BCD6552750C12124B4BDDB76D7461894
:10DB100038DF5438DF5218D64686209046270F78D3
:10DB200000557900547900537900524A20EF7B80E8
:10DB3000522705720403200371FB0372041571FB65
:10DB4000157800557900547900537900525A26DE31
:10DB500072201571DF157EEDFEC60849240572049A
:10DB600003200371FB0372041571FB155A26EC7236
:10DB7000201571DF153986049A8A9701978A8624C1
:10DB80009A8B9720978B71DB15398627BDEDE72798
:10DB90000A8622BDEDE727037EF2C2BDDBC6974EA3
:10DBA000BDDBC636BDDBC61632DD46BDDBC6BDDB22
:10DBB000C6D64E270E5AD74E3CDE46A70008DF4693
:10DBC0003820EB7EEDFE8D0A48484848368D0333F9
:10DBD0001B39A600088030250C810A250B800725FB
:10DBE00004811025037EF2C239CC00217EEF0B7E2A
:10DBF000F2C2BDE2DFDC5226F0DC54183C18862C61
:10DC0000BDEDE726EABDEDF7812227048127261026
:10DC1000183818DDACBDCC6ACCF8F3DDAC7EEDFE77
:10DC2000BDE2DF18DE523CDE543C18862CBDEDE729
:10DC30002705CC004E2005BDEE0425B3FD73AA18C0
:10DC400038DF5438DF5238DF46183CBDF88126FBF8
:10DC5000CEDC5C3CDE463CDC54DE52393CFE73AA32
:10DC6000ED02183818ED00387EEDFE7EF2C238CC99
:10DC700000247EEF0BBDEE0425F13C188C719C2531
:10DC8000EDEC00DD56EC02DD54188372184353C3EB
:10DC90000001541736BDF6AFDC54DD56324CBDF6EC
:10DCA000AF387EEDFE7EF2C238CC00247EEF0BBD95
:10DCB000EE0425F13C188C719C25ED3C18837218FC
:10DCC0004050C30001541736BDF65FDC56DD5232BA
:10DCD0004CBDF65F38DC56ED02DC52ED00387EEDCF
:10DCE000FEBDE52BDC522615DC54188C0014250CE7
:10DCF0008C0C01240718FD72887EEDFE18CC0023E1
:10DD00007EEF0B7F00B37F00B4867BBDEDE7260E70
:10DD1000BDEE04250CDDB3867DBDEDE726037EED6B
:10DD2000FE7EF2C27F0008BDEE04251CFDB598867C
:10DD30007EB70109CCDD4BFD010AC602D708D60823
:10DD4000DC0DDC09C612D7087EEDFE9608FEB598FC
:10DD5000EC02C30001ED02EC00C9008900ED00DE19
:10DD60000D3B86FF974F860197503CCC0052FD73C8
:10DD7000ACBDEE0425123637862CBDEDE726073301
:10DD800032FD73AC2002323338BDE2DFDC52DD6499
:10DD9000DC54DD66862CBDEDE727037EF2C2BDEEC6
:10DDA0000425F8FD73AA3C96B636861897B6BDF8DA
:10DDB00054CE006496431A914327F9BDF87C26EEB1
:10DDC0000926F18615BDF8F37C004FD64FC1142605
:10DDD000208618BDF8F3FE73AA4FED025FED00FE3A
:10DDE00073ACDC66ED02DC64ED003297B6387EED94
:10DDF000FEBDDE7627CDBDF8B681182604C61520F7
:10DE0000D5810426098606BDF8F3D64F20C88101C6
:10DE1000269CBDDE2126978606BDF8F37C005020A7
:10DE2000D0CEB394C683BDDE66A700085A26F7FCA1
:10DE3000B3945311270139CEB3964FAB00088CB47D
:10DE40001626F8B1B416270139B6B3944C91502672
:10DE5000064A9150270139CEB396A600BDEFD508EA
:10DE60008CB41626F5393CBDDE76382704BDF8B6ED
:10DE70003938387EDDAECE01F4BDF87C2701399605
:10DE8000431A914327F90926F03938CC00017EEF77
:10DE90000B7EF2C2BDEE04240ABDEE6C964427F15F
:10DEA000CC0052FD73AA3C18EC0026DEEC02FD7398
:10DEB000AC38862CBDEDE726D87EDED0863BBDEDA6
:10DEC000E727F63CFE73AAFC73ACED02387EEDFE4C
:10DED000CCE0FDDD46BDEDF7DF483CDE46A1002687
:10DEE0000908DF463808A60020F0A6002B1908A66E
:10DEF000002AFB0808A6002604387EF2C2DF463856
:10DF0000DE48A6007EDEDA3C16584FC3E0E718EC88
:10DF100000186E0038A601BDE0DB387EDEBC38A6F6
:10DF200001BDE0DB38BDE2DFDC5227037EEF0BDC16
:10DF3000542718830001B373AC4D2606C18024EC2E
:10DF4000200881FF26E6C18025E217BDE0DB7EDEEA
:10DF5000BC38A60138E600C1412706C14226058B20
:10DF6000100820E736BDE2DFBDE0A2270C328B307F
:10DF7000BDE0DBBDE0BC7EDEBC32BBC431BDE0DB5E
:10DF8000BDE0C77EDEBC38A6013836BDE2DFDC521C
:10DF900027037EEF0BDC544D26F837862CBDEDE7CA
:10DFA00027037EF2C2BDE2DFDC5226E6DC544D26BA
:10DFB000E1BDE0A22616DF46183332BDE0DB17BD17
:10DFC000E0DB1817BDE0DBDE467EDEBCDF46183343
:10DFD000328B107EDFBB38A601387EDF6438A601A5
:10DFE00038E600C1412709C14227037EF2C28B40B7
:10DFF00036088623BDEDE7262EBDE2DF32BDE0DB2D
:10E00000BDE0C77EDEBC38A6013836B6C42D802BF5
:10E01000BDEDE72612BDE2DF32BDE0DBBDE0BC7E38
:10E02000DEBC38A6013836BDE2DFBDE0A2260C32E8
:10E030008B20BDE0DBBDE0C77EDEBC9654270C32F2
:10E040008B30BDE0DBBDE0BC7EDEBC328B1020E25D
:10E0500038A601BDE0DB38BDE2DFBDE0C77EDEBC37
:10E0600038388622BDEDE72604167EE0758627A1A6
:10E0700000260D1608A6000811270BBDE0DB20F5D1
:10E08000BDE2DFBDE0C7862CBDEDE727D57EDEBC57
:10E090003838BDE2DFBDE0BC862CBDEDE727F37E5E
:10E0A000DEBCA600B1C42B26030820F6812C260B6B
:10E0B00008A60008815827037EF2C239DC52260EDA
:10E0C0009654BDE0DB200EDC522706CC00277EEF05
:10E0D0000B965426F99655BDE0DB393CFE73ACA790
:10E0E0000008FF73AC3839DF14DF1EDF51DF86DF35
:10E0F000D6DFDDE006E022E050E060E0904E4F50D9
:10E1000080014C535244800441534C448005544197
:10E110005080065450418007494E58800844455865
:10E120008009434C56800A534556800B434C43802C
:10E130000C534543800D434C49800E534549800F95
:10E140005342418010434241801154414280165451
:10E150004241801758474458801844414180195320
:10E160004C50801A414241801B5453588030494ED4
:10E1700053803150554C41803250554C428033448D
:10E18000455380345458538035505348418036505D
:10E19000534842803750554C588038525453803938
:10E1A000414258803A525449803B50534858803C31
:10E1B0004D554C803D574149803E535749803F4221
:10E1C0005241812042524E81214248498122424C93
:10E1D00053812342434381244243538125424E4588
:10E1E0008126424551812742564381284256538118
:10E1F0002942504C812A424D49812B424745812C6E
:10E20000424C54812D424754812E424C45812F4E21
:10E2100045478240434F4D82434C53528244524FB4
:10E22000528246415352824741534C8248524F4C8E
:10E230008249444543824A494E43824C5453548256
:10E240004D434C52824F41494D83614F494D83624A
:10E2500045494D836554494D836B4A4D50844E5317
:10E2600055424486834144444486C3435058868C77
:10E270004C444486CC4C4453868E4C445886CE53F2
:10E2800055428580434D5085815342438582414E9E
:10E2900044858442495485854C44418586454F5286
:10E2A000858841444385894F5241858A414444854C
:10E2B0008B5354414187875354414287C75354532A
:10E2C000878F4A5352878D53544487CD5354588770
:10E2D000CF425352888D4442890044578A0000BD82
:10E2E000E30FF6C431A600081127FA817C27020942
:10E2F00039DC543736DC523736BDE30F32339A52AD
:10E30000DA53DD5232339A54DA55DD547EE2E2BDFF
:10E31000E33FF6C42BA600081127FA81262702093D
:10E3200039DC543736DC523736BDE33F3233945252
:10E33000D453DD5232339454D455DD547EE312BDB0
:10E34000E3E5A60008B1C43A27F809813C25048119
:10E350003F250139DC543736DC523736CCC649DD2F
:10E36000527EC866BDE3AA250B860197552008BDDD
:10E37000E3AA26F57F00557F00547F00537F0052AB
:10E3800039BDE3AA27EE25EC20DFBDE3AA27DA2575
:10E39000D820E1BDE3AA26DC20CFBDE3AA24D52006
:10E3A000C83233DD523233DD5439DF4E381838DFAE
:10E3B0005038183C183CDE503CDE4EBDE3E53233AD
:10E3C000DD463233DD4896469852182A0CDE529CC0
:10E3D000462610DE549C481839DE469C522604DE40
:10E3E000489C541839862DBDEDE72606BDEF8A7E80
:10E3F000E43E862BBDEDE7BDE44F862BBDEDE72661
:10E4000035DC543736DC523736BDE44F3233DD4627
:10E410003233DD48DC54D348DD54DC52974ED947C3
:10E420009946DD52964E98462BD0964E98522ACA5F
:10E43000CC00097EEF0B862DBDEDE7270139DC54BA
:10E440003736DC523736BDE44FBDEF727EE40CBD8B
:10E45000E4E3862ABDEDE72621DC523637DC54366C
:10E4600037BDE4E33332DD483332DD46BDF160DCF5
:10E470004EDD52DC50DD547EE452A600812F27058C
:10E4800081252701393C087F00447D00522A067C03
:10E490000044BDEF72DC523637DC543637964436D2
:10E4A000BDE4E33297447D00522A067A0044BDEF72
:10E4B00072DC52DD46DC54DD483332DD543332DD6C
:10E4C000523CBDF08238183836A60081252608DE79
:10E4D0004EDF52DE50DF54321896442703BDEF72F0
:10E4E0007EE4520908A600812027F98130250481A5
:10E4F0003A25308128273E81262728A601814125FB
:10E500000C815B2408CCC5BFDD527EC866BDEE041D
:10E51000DD52251E3C0FDE52EC00DD52EC020EDD1A
:10E52000543839BDEE6C96442708398628BDEDE78E
:10E5300027047EF2C208BDE2DF8629BDEDE726F2A0
:10E5400039BDE52B96522A03BDEF7296522B013945
:10E55000CC000A7EEF0BBDE52BDC522706CC000B6E
:10E560007EEF0B3C8D0738DD545FDD5239DE548C75
:10E570000008250A9D9F3838CC000B7EEF0B18C38E
:10E58000E58A18E600BDF7124F391F1B1E1A1D1928
:10E590001C1818FE73AA3CDE643CDE663C18862814
:10E5A000BDEDE72629BDCF517F00527F00537F008C
:10E5B00054862CBDEDE726288623BDEDE7260FA661
:10E5C00000088134270B81322711813127127EF216
:10E5D000C2BDF0409752BDF0409753BDF0409754F4
:10E5E000BDF04097553CFE73AADC66ED02DC64ED9D
:10E5F00000381838DF6638DF6438FF73AA188629B8
:10E60000BDEDE726C9399DA23838CC000C7EEF0B52
:10E610008628BDEDE72657BDEF8ADC54053736BDA9
:10E62000E2DFDC52270CCC000C7EEF0B3C8DD738A0
:10E630002021DC544D26F5C10E24F1C10824338677
:10E64000805D2704445A20F93643948B9720978B9A
:10E6500032941527073233C3000120023233DD54D0
:10E66000862CBDEDE727B38629BDEDE727037EF2B3
:10E67000C239C00886805D2704445A20F9B1C43AE3
:10E68000240244443643948A9701978A32940320A3
:10E69000C2BDE52B96522A06CC000D7EEF0BCC00B6
:10E6A00000DD46DD48DD4EDD50DD4CCC4000DD4A6E
:10E6B000860F975ADC48D350DD58DC46D94F994E27
:10E6C000DD56DC58D34CDD58DC56D94B994ADD5623
:10E6D00074004E76004F760050760051DC5293560F
:10E6E000251E2606DC5493582516DC56DD46DC58DC
:10E6F000DD48DC50D34CDD50DC4ED94B994ADD4E21
:10E7000074004A76004B76004C76004D74004A76D1
:10E71000004B76004C76004D7D005A2609DC4EDD1C
:10E7200052DC50DD54397A005A20893CBDEF8AC64C
:10E730001CBDF712D7547F00467F0047CC028DDD09
:10E7400048BDF0823839BDE52BDC522706CC000EDF
:10E750007EEF0BDC544D26F517C4FC105497464F42
:10E76000C3E7853C18EC00DD4EA30296463DCB0284
:10E7700004044353C30001D34EDD542A06730052F0
:10E78000730053383905DC05DC055A04AB04360345
:10E79000DF038E0353032102F402CD02A902880293
:10E7A0006A024E0233021A020301EC01D701C201D0
:10E7B000AE019B01890176016501540143013201DB
:10E7C000220112010200F200E200D300C400B400F2
:10E7D000A4009500850076006600560046003500CE
:10E7E0002400130001FFEEFFDCFFC8FFB3FF9DFF15
:10E7F00086FF6DFF53FF35FF15FEF0FEC4FE8FFE52
:10E8000048FE1BFE1BFE1BBDE52B3C7D00522A096A
:10E81000DC545343C38001DD54DC54847FDD521843
:10E820008C4000182505CC80009352DD46164F051C
:10E83000C3E8DC18EC00DD48EC02A300974E9647D5
:10E840003D97517F0050D64E96473DD350D3487FD9
:10E8500000527F00537D00542A15435373005273B6
:10E860000053C3000118DC52C9008900DD5218DDD5
:10E87000543839BDE52B3C7F00567D00522A06BD39
:10E88000EF727A0056DC52270738CC000F7EEF0B70
:10E89000DC5427462BF3CEE8DC7F0057EC00189CB5
:10E8A0005418240708087C005720F1DD4A0909ECB8
:10E8B00000DD4CDC4A934CDD48CE0000DF46DC54E2
:10E8C000934CDD537F0055BDF08296574A5FD35479
:10E8D000DD547D00562703BDEF7238390000032454
:10E8E0000648096A0C8C0FAB12C815E218F91C0B0C
:10E8F0001F1A2223252828262B1F2E1030FB33DE3B
:10E9000036BA398C3C563F1741CE447A471C49B43D
:10E910004C3F4EBF5133539A55F558425A825CB31F
:10E920005ED760EB62F164E866CF68A66A6D6C231F
:10E930006DC96F5E70E2725473B575047641776B82
:10E94000788479897A7C7B5C7C297CE37D897E1D57
:10E950007E9C7F097F617FA67FD87FF57FFFCC00FB
:10E9600002DD545FDD5239FCFFE8DD547F00527F49
:10E970000053393CCEC403BDEE6C3839CC00107E58
:10E98000EF0BBDE52BDC5226F3965426EFD655BD92
:10E99000EF8A5D27E7C12124E386BF948A97019718
:10E9A0008A968B8A14978B972071EB15721015201D
:10E9B0001278005579005479005379005272041589
:10E9C00071FB157B400327037C00555A26E339CCA5
:10E9D00000117EEF0BBDE52BDC5226F3DC54274003
:10E9E0003C18968A84FE9701978A867EB70109CCE7
:10E9F000EA21FD010A7F00547F005596431A914396
:10EA000027FB01010101D608DC0D9643C6120FD782
:10EA1000080E1A914327F796430926F27F0008381B
:10EA200039960884EF9708DC0DDC54C30001DD54EF
:10EA3000DC52C9008900DD523B9608DE4A08DF4AF5
:10EA400084E29708DE0DDF54B4C42B270EDE548C0D
:10EA500080002407DE5208DF52DC093B960820F4D0
:10EA60007EF2C2CC00127EEF0B8628BDEDE726F0C9
:10EA7000BDE2DFDC5226ECDC5427E8183C18862C7B
:10EA8000BDEDE726DBBDE2DFDC5226D7DC5427D321
:10EA9000DD4E183818DD508629BDEDE726C23C96BC
:10EAA0008A84FE9701978A867EB70109CCEA39FDF0
:10EAB000010A867EB70103CCEA5CFD01047F004AAF
:10EAC0007F004B7F004CC602D708CC0000DC09D683
:10EAD00008DC0DDC099643C6160FD7080E1A9143C1
:10EAE00027099643DE4E092731DF4E0FDE4A0926FD
:10EAF00011964C260D7C004CDE52DF46DE54DF487A
:10EB000020D79C5026D30E7F0008DC549348DD5458
:10EB1000DC52D2479246DD5238397F0008CC0000E3
:10EB2000DD52DD543839BDE52B7F005ADC522A0610
:10EB3000CC00137EEF0B3C27157400527600537601
:10EB400000547600557C005ADC5226ED2011DC542E
:10EB500027DE2B0B7800557900547A005A20EF7F7E
:10EB600000467F0047DC54C3B172DD487C0047CCCF
:10EB7000B172DD52CC17ADDD54BDF082DC54DD56F0
:10EB80007F0058DC4FDD52965197547F0055BDF001
:10EB900082DC54D357DD5796568900975696568097
:10EBA000809756DC5805DD58DC565949DD56730010
:10EBB00056DC574353C30001DD57965689009756DC
:10EBC000CE0000DC56DD54DD482A03CEFFFFDF52C5
:10EBD000DF46BDF160DC4EDD5EDD54CC994BDD4897
:10EBE000CC0000DD46DD52BDF160DC4EC3F622DD17
:10EBF00054DC5EDD48CC0000DD52DD46BDF160DC5A
:10EC00004EC3E2A8DD60CC0002DD5EDC57DD544F70
:10EC1000D6562A0286FFDD52DC54363705DD58DC35
:10EC20005236375949DD56CC0000DD46974896608C
:10EC30009749BDF160DC4FD358DD58DC56C90089D7
:10EC400000DD564FD64E2A0286FFD356DD56D661DA
:10EC5000D7493332DD523332DD54BDF160DC4ED35F
:10EC600058DD58DC56C9008900DD564F5F7D004EE7
:10EC70002A03CCFFFFD356DD56DC5783875DDD5377
:10EC80009656820097524F965A9B529752DC53DD0C
:10EC90005436374FD6522A0286FF3637DD5286B1B8
:10ECA0009749CC0000DD469748BDF160DC4EDD564B
:10ECB000DC50DD58C672D7493332DD523332DD5471
:10ECC000BDF160DC4ED357DD548600D6562A02864D
:10ECD000FFC90089007D004E2A03C3FFFFDD5238C3
:10ECE00039BDE52BDC522B0B83000A2506CC001422
:10ECF0007EEF0BDC52DD56DC54DD58DC53DD5496E0
:10ED0000529753CC0001DD46CC62E4DD48BDF16092
:10ED1000D64E2A0CC1F02408CC0000DD52DD543957
:10ED20004F5CD75A2A0286FFDD5416DD52CCB172F1
:10ED3000DD487F00467F0047BDF160DC509358DD21
:10ED400054DC4ED2579256DD52DC524756DD5EDC23
:10ED5000544656DD608607975B3CCCFFFFDD52CC06
:10ED6000FFF3DD54CEEDCBBDED977A005B26F89630
:10ED70005A2B13270F7800557900547900537900E6
:10ED8000524A26F13839770052760053760054768D
:10ED900000554C26F13839DC5EDD46DC60DD48BDCF
:10EDA000F160965048DC4E5949DD54CC00007D009E
:10EDB0004E2A03CCFFFFDD52EC02D354DD54EC00AD
:10EDC000D9539952DD5208080808390000005BFF4A
:10EDD000FFFDDE00000AABFFFFD55500008000FFFD
:10EDE000FF000000010000160908A600812027F995
:10EDF00008112701093908A600812027F939BDF239
:10EE00009D7EF2C20908A600812027F9813F2626AF
:10EE100008A600812027F981282705CC00400C395D
:10EE2000BDE52BDC522627DC544D2622C106241ECC
:10EE30000505C373B0398040240139262008BDE59B
:10EE40002BDC522609DC5418BC7288182506CC002D
:10EE5000027EEF0B05054353C372190C39811B2544
:10EE6000020D39084848164FC3721839BDEF8A7F22
:10EE70000044BDEDF77F0046812626037EEF2C81FE
:10EE800030240139813A250139840F7D0044260A56
:10EE90007C0044975508A60020E57C0044D644C178
:10EEA0000524149747DC5405DD540505D354D34697
:10EEB000DD5408A60020C89747DC5405DD54DD501A
:10EEC000DC5259492B42DD52DD4E78005179005019
:10EED00079004F79004E2B3078005179005079003D
:10EEE0004F79004E2B22DC54D350DD54DC52D94FE5
:10EEF000994E2B14DD52DC54D346DD54DC52C9004C
:10EF000089002B04DD5220AACC00033CCEEF127EF8
:10EF1000F2C8484F573F20204552524F52202300FD
:10EF2000574841543F0D534F5252590D08A6008186
:10EF300048270909399644260209093908A600809C
:10EF40003025F2810A250A8007810A25E8811024EC
:10EF5000E47C0044D644C10924AEC6047800557947
:10EF600000547900537900525A26F19B5597557EEB
:10EF7000EF3C730052730053DC544353C30001DD74
:10EF800054DC52C9008900DD52397F00527F0053A2
:10EF90007F00547F0055393CFE738C3CCEEFBFFFA1
:10EFA000738CBDEFD538FF738C38393CFE738C3CC5
:10EFB000CEEFBFFF738CBDF04038FF738C38390043
:10EFC00001004441544146494C45204F5645525258
:10EFD000414E4745003CBDEFDB3839367D006426A5
:10EFE00009DC650525048101250B329D943838CC58
:10EFF00000047EEF0B331807360F1837D617C4F806
:10F000001B4C330F308C010125059F688E00FF9744
:10F010001737DC66847FC340001832A700D617C4B8
:10F02000F8D717308C010026029E6816320637DCAE
:10F0300066C30001DD66DC64C9008900DD64323925
:10F040003CBDF04638397D00642609DC65052504A1
:10F050008101250A9D973838CC00057EEF0B1607F5
:10F060003617D617C4F81B4C0F308C010125059FAD
:10F07000688E00FF9717DC66847FC3400018A600E7
:10F08000209BDE46264BDE4826083838CC00067E1C
:10F09000EF0BDE52263BDC54CE00007C00527800A1
:10F0A0004979004824F576004876004993482404BD
:10F0B000D3482001087A0052270B1805187400481D
:10F0C00076004920E7DF54CE0000DF52DF4EDD50EE
:10F0D000397F004ADE52DF4EDE54DF50CE0000DFC3
:10F0E00052DF547C004A780049790048790047791A
:10F0F000004624EF760046760047760048760049C1
:10F10000DC509348DD50DC4ED2479246DD4E241051
:10F11000DC50D348DD50DC4ED9479946DD4E2012F5
:10F120007C0055240D7C005424087C005324037C6F
:10F1300000527A004A271A78005579005479005312
:10F1400079005274004676004776004876004920E0
:10F15000AF393CCE004686106F00084A24FA383991
:10F160007F00447D00522A067C0044BDEF727D0082
:10F17000462A1A7A0044730046730047DC4843531A
:10F18000C30001DD48DC46C9008900DD46BDF1B69B
:10F19000964E2A06CC00077EEF0B96442717730085
:10F1A0004E73004FDC504353C30001DD50DC4EC9A9
:10F1B000008900DD4E397F004E7F004F9649D655BD
:10F1C0003DDD50D655272F9648270B3DD34FDD4FB9
:10F1D000964E8900974ED6559647270A3DD34EDD69
:10F1E0004E24037EF274D6559646270A3D4D26F3EB
:10F1F000DB4E25EFD74ED65427389649270B3DD303
:10F200004FDD4F964E8900974ED654964827083DBD
:10F210004DD34E25CEDD4EF6C42FC1452614D6540F
:10F220009647270A3D4D26BBDB4E25B7D74E96465F
:10F2300026B1D6532723964927093DD34EDD4E25C7
:10F2400033974ED6539648270A3D4D2627DB4E2549
:10F2500023D74E96479A46261BD6522716964927FD
:10F260000A3D4D260FDB4E250BD74E96489A479AFE
:10F2700046260139CC00077EEF0BBDEE042543374F
:10F2800036863DBDEDE7263ABDE2DFDF46380FDCCE
:10F2900052ED00DC54ED020EDF52DE4639863ABDF7
:10F2A000EDE7260532327ECAF5860DBDEDE726066E
:10F2B0003232087ECABF39BDEDF7810D27F8813A99
:10F2C00027F43C4F5FCEEF200EDD547F00527F00CD
:10F2D00053CCF8F3DDAC7F00B57D008127273CFEE1
:10F2E000738C8CFFFF38271D96B681182606BDF853
:10F2F000F37F00B68EBFFFCC0000FD738EFD7394CC
:10F30000DE82BDCACD7F00B37F00B496B6270CBDA8
:10F31000F8F396B6811826037F00B64FBDF46086D9
:10F320000AB7B59ADC5427097F0045BDF49BBDF5AB
:10F33000DFFE738C8CFFFF26037ECDD5EC00260309
:10F340007EC6FEBDF535183809DF4618A600810DCA
:10F35000270FBDF5E19C462605863FBDF5E1082057
:10F36000EBBDF5E17EC6FE3CCEEF264F5F7EF2C8D8
:10F37000C60DD74636DF5218C300F0DD54DE52BD4D
:10F38000F8B6817F27418108273D810A27F1810056
:10F3900027ED810326113337C13A260B333838382D
:10F3A000FF738C387EF602A700089146261233C1FF
:10F3B0003A270CBDF8F3810D2605860ABDF8F3390E
:10F3C000BDF8F39C5426B89C5227B4098608BDF8B2
:10F3D000F38620BDF8F38608BDF8F320A2DE548C36
:10F3E00080002508CC00087EEF0B3232CE73D2BCF1
:10F3F00073A225040D86FF39EC00847F9354250108
:10F4000039E602DF564FD3561820E4200108A60043
:10F410002AFB20DB3CDE52270738CC00087EEF0BAE
:10F42000DE548C800024F2FE738CEC00847F260373
:10F430005D27B7189C543825D2FE738C200C09E642
:10F44000000886FF50DF56D35618DC548A80A1008E
:10F450002605E1012601398C73D226E20D86FF399B
:10F4600016A60008112601393637BDF5E133328181
:10F470000D26EE398622BDEDE7260ABDF460810D2A
:10F480002601094F398627BDEDE727EF817F260A40
:10F4900081082606860D9DAB20E9393C96453684C9
:10F4A0008097449645847F97458614367A0045F6C2
:10F4B000B59AC10A260E7D00522A09BDEF727C0062
:10F4C000447A0045F6B59A4F18DF487F00477F0021
:10F4D00046BDF082DE522604DE542708D651377A24
:10F4E000004520E0D651377B80442715964484019F
:10F4F0002704862D9DAB7A00452B1B86309DAB20C3
:10F50000F57A00452B0686209DAB20F596448401B4
:10F510002704862D9DAB328114270C810A25028B8E
:10F52000078B309DAB20EF3297453839BDF5354F0D
:10F53000BDF4600839EC00847FDD547F00527F0009
:10F540005308080886049745BDF49B8620BDF5E165
:10F5500039FE73A4BC73A8260139A600083CFE73CB
:10F56000A6A70008FF73A63820EAFE73AABC73AEF4
:10F5700026013909A6003CFE73AC09A700FF73AC55
:10F580003820EA3233DF5E38FF7394271838FF7370
:10F590009A38FF739C38FF739638FF739838FF735F
:10F5A0009E38FF73A03736DE5E393233DF5E308C33
:10F5B000B6012405DE5E7EF367FE7394271BFE739F
:10F5C000A03CFE739E3CFE73983CFE73963CFE731B
:10F5D0009C3CFE739A3CFE73943C3736DE5E398663
:10F5E0000D369DAB3236810D2604860A9DAB32392D
:10F5F0007D00932601397D009E27FA7F0093BDF898
:10F60000540E7D008C271A8EBFFDCC0000FD738E3A
:10F61000FD7394CC0064DD54CC0000DD523C7ECB05
:10F6200004FE738C2727CEF650BDF5DF4FBDF46086
:10F63000FE738CEC00847FDD547F00527F00537F8B
:10F640000045860AB7B59ABDF49BBDF5DF7EC6FEC0
:10F65000425245414B204154204C494E4520000F19
:10F6600036BDF75C32843F8A8016BDF691C6EFD76F
:10F670001671DF17BDF763D756BDF763D757BDF7D0
:10F6800053C6FFD7160E39BDF69171DF1771BF173C
:10F690003971DF1771BF1771EF177240177220179A
:10F6A00071DF177210177220178608BDF786390FA1
:10F6B00036BDF75C32843F36C630BDF68732368AB7
:10F6C000C016BDF691BDF6EC0E01010F32843F8AE3
:10F6D0004016BDF691D656BDF784D657BDF784BD0A
:10F6E000F6ECC600BDF687BDF7530E3971EF177102
:10F6F000DF1771BF17CE026272201701010101717D
:10F70000DF170926F372401772201771DF1771BFD8
:10F710001739B6C4308154270AC11C2706C11827DF
:10F7200002D643BDF75CBDF72DBDF753390F9F6877
:10F730008E00FF71BF177220175858588605BDF705
:10F7400086C6EFD71671DF17BDF76386FF97169E43
:10F75000680E399617840F8A80971739710F1772C0
:10F76000401739C60272201771DF177B1017270167
:10F770005C7220175824F171DF177B101727015C8A
:10F780007220173986085871DF1772101725037118
:10F79000EF177220174A26EE39961ED6113784D0FD
:10F7A0002756845027049612323BDE719612A7002A
:10F7B0007B0176271281132605728076203A81110B
:10F7C0002605717F762031810326037C0093098C06
:10F7D000728B2603CE738BDF717D0075261A18930A
:10F7E00073C1402613FCB596B3B594C1FF270986B3
:10F7F00013BDF8F386FF9775328424812427013BDB
:10F800007B017627237B8076271EDEAFBDF5F07166
:10F81000FB110E010196431A914327F90F092705A1
:10F820007B807626E7717F76FEB596A600098CB4BC
:10F83000932603CEB593FFB5967D007726029713E6
:10F84000FEB596BCB594260471FB113B7204113BC6
:10F8500086FF97753CCE738BDF71DF7371FB11CE22
:10F86000B593FFB594FFB596967527088611BDF838
:10F87000F37F007538717F767F00933996749072AC
:10F8800039B6B597B0B59539DE643CDE663CDEB37B
:10F89000EC00DD64EC02DD663CBDF04038D664E788
:10F8A00000D665E701D666E702D667E70338DF666C
:10F8B00038DF643338393C3736DCB33226CADE737E
:10F8C0009C7126031A20F7A60036098C728B26033A
:10F8D000CE738BDF739675270F189371C14026087E
:10F8E0008611BDF8F37F0075323338810326037A21
:10F8F0000093393C3736FCB596B3B594C1FF27F673
:10F90000FEB59432A700098CB4932603CEB593FFBD
:10F91000B59472041133383986209DAB86209DAB97
:10F92000393B3B717F1BDE6C08DF6CDC42C300019E
:10F93000DD42DC40C9008900DD4096AE890097AE0B
:10F940003B7B201127FB971339860297908E00FD91
:10F95000BDF9631A1A1ACE0000DF42DF407F00AE05
:10F960007EC6838612971BB6C42E8B0C971C97639A
:10F970007F00017F00207F008B7F008A860A97111D
:10F980008605971086E097148680971786029790D1
:10F9900086FF9716860397707F009186FF97808673
:10F9A0007EB7010FCCF923FD011072401B0E86FFBC
:10F9B0009777392A202050433D2420413D2420427E
:10F9C0003D2420463D2420583D242040583D2420FD
:10F9D00053503D24204024DEAC3CCEF8F3DFAC0E87
:10F9E000860DBDF8F3860ABDF8F3CEF9B3BDFA6F04
:10F9F0003C30EC091809BDFA7738BDFA6F3C30A6E7
:10FA000006BDFA7C38BDFA6F3C30A605BDFA7C38DD
:10FA1000BDFA6F3C30A604BDFA7C38BDFA6F3C30AD
:10FA2000EC0718BDFA7738BDFA6F3C30EC0718ECDC
:10FA30000018BDFA7738BDFA6F3C3018C3000A18B9
:10FA4000BDFA7738BDFA6FFE7282BDFA77863DBD8A
:10FA5000F8F3FE7282860836A60008BDFA7C86207E
:10FA6000BDF8F3324A26F038DFAC3BBDF8F308A608
:10FA700000812426F608393C328D01323644444454
:10FA8000448D0132840F8B30813A25028B077EF83A
:01FA9000F382
:10FFCA007EF72D7EF75C7EF7537EEF977EEFAB7E52
:10FFDA00F87C7EF8B67EF8F37EF8547EF71200C3FA
:10FFEA000100010FF921F799010301060109010C2A
:06FFFA00F9D7F922F949D4
:00000001FF
